:100000000C94300018950000189500001895000019
:10001000189500001895000018950000189500002C
:10002000189500001895000018950000189500001C
:10003000189500001895000018950000189500000C
:1000400018950000189500001895000018950000FC
:1000500018950000189500001895000018950000EC
:100060008FE181BD87E181BD8FEF8DBFC0EEEEEBEB
:100070004E2E8FE08EBFDFE0FFE05F2EEEE9FFE067
:10008000A0E6B0E088278D933197E9F785B7806CBB
:1000900085BF89E189B988E18AB90E94B90A6624D5
:1000A000B89AB99ABA9ABB988CE291E00E94E60A93
:1000B0000E94CF0A0E94B5005A924A928EEBA42D5C
:1000C000B52D8C9381E00E94880A5A924A9200E0F2
:1000D00010E020E030E0A42DB52D0D931D932D935D
:1000E0003C9384E00E94880A0E943B07249685E0A6
:1000F0000E94840A5A924A9200E010E020E030E028
:10010000A42DB52D0D931D932D933C9384E00E9457
:10011000880A0E949F02229684E00E94840A0E941C
:100120005B0AC09ABA9AB99AC19AA0E7B2E011964E
:1001300098E08E91983018F4392F992702C038E052
:100140009850881FC29808F4C29A00000000C19815
:1001500000000000C19A000000003A9591F7992331
:1001600041F70C94B100F894FFCFC09A8FEF8093C1
:10017000700281E090E0A4E7B2E08D939C93A4E745
:10018000B2E00D911C910A3050E0150718F011F003
:100190000C94F000BA9AB99AC19AA0E7B2E011960D
:1001A00098E08E91983018F4392F992702C038E0E2
:1001B0009850881FC29808F4C29A00000000C198A5
:1001C00000000000C19A000000003A9591F79923C1
:1001D00041F7A4E7B2E00E948C0A11F00C94BF0032
:1001E0008FEF80937102C09880E480937002BA9A76
:1001F000B99AC19AA0E7B2E0119698E08E91983032
:1002000018F4392F992702C038E09850881FC298F7
:1002100008F4C29A00000000C19800000000C19AD2
:10022000000000003A9591F7992341F700E010E0B3
:1002300020E030E0A0E8B2E00D931D932D933C93B5
:10024000BA9AB99AC19AA0E8B2E0149690E28E9157
:10025000983018F4392F992702C038E09850881F39
:10026000C29808F4C29A00000000C1980000000083
:10027000C19A000000003A9591F7992341F785E96A
:1002800080937002BA9AB99AC19AA0E7B2E0119627
:1002900098E08E91983018F4392F992702C038E0F1
:1002A0009850881FC29808F4C29A00000000C198B4
:1002B00000000000C19A000000003A9591F79923D0
:1002C00041F700917102013011F40C948601B99A42
:1002D000BB98C19A98E0A1E7B2E01196983018F463
:1002E000392F992702C038E09850C19800000000CB
:1002F0008894B3990894881FC19A000000003A9529
:10030000A1F78E93992351F70C946101E4E3F6E190
:100310000E94FB0A0E94B00AAEEABFE0E1E7F2E009
:100320000E94FE0A0E94A80AC09A82E390E00E94FE
:10033000E60AC0988FEF809370020091710200303E
:1003400011F40C948C02C09ABA9AB99AC19AA0E797
:10035000B2E0119698E08E91983018F4392F9927D1
:1003600002C038E09850881FC29808F4C29A000072
:100370000000C19800000000C19A000000003A95FA
:1003800091F7992341F7B99ABB98C19A98E0A1E7F0
:10039000B2E01196983018F4392F992702C038E04E
:1003A0009850C198000000008894B3990894881F61
:1003B000C19A000000003A95A1F78E93992351F756
:1003C000C09881E480937002BA9AB99AC19AA0E762
:1003D000B2E0119698E08E91983018F4392F992751
:1003E00002C038E09850881FC29808F4C29A0000F2
:1003F0000000C19800000000C19A000000003A957A
:1004000091F7992341F700E010E020E030E0A0E808
:10041000B2E00D931D932D933C93BA9AB99AC19A69
:10042000A0E8B2E0149690E28E91983018F4392F3B
:10043000992702C038E09850881FC29808F4C29AE1
:1004400000000000C19800000000C19A00000000F8
:100450003A9591F7992341F78FEF80937002BA9AFA
:10046000B99AC19AA0E7B2E0119698E08E919830BF
:1004700018F4392F992702C038E09850881FC29885
:1004800008F4C29A00000000C19800000000C19A60
:10049000000000003A9591F7992341F7BA9AB99A6A
:1004A000C19AA0E7B2E0119698E08E91983018F4C6
:1004B000392F992702C038E09850881FC29808F455
:1004C000C29A00000000C19800000000C19A00001C
:1004D00000003A9591F7992341F7B99ABB98C19AD0
:1004E00098E0A1E7B2E01196983018F4392F9927D7
:1004F00002C038E09850C198000000008894B39979
:100500000894881FC19A000000003A95A1F78E93C5
:10051000992351F70C949D018FEF80937002C09A3C
:10052000E8E3F6E10E94FB0A0E94B00AAEEABFE0EF
:10053000E1E7F2E00E94FE0A0E94A80A0895C09A2C
:100540008FEF80937002BA9AB99AC19AA0E7B2E08D
:10055000119698E08E91983018F4392F992702C09F
:1005600038E09850881FC29808F4C29A0000000032
:10057000C19800000000C19A000000003A9591F770
:10058000992341F7B99ABB98C19A98E0A1E7B2E0E4
:100590001196983018F4392F992702C038E09850F6
:1005A000C198000000008894B3990894881FC19AEC
:1005B000000000003A95A1F78E93992351F7C09857
:1005C00081E580937002BA9AB99AC19AA0E7B2E025
:1005D000119698E08E91983018F4392F992702C01F
:1005E00038E09850881FC29808F4C29A00000000B2
:1005F000C19800000000C19A000000003A9591F7F0
:10060000992341F7BA9AB99AC19AA881B9811496E7
:1006100090E28E91983018F4392F992702C038E073
:100620009850881FC29808F4C29A00000000C19830
:1006300000000000C19A000000003A9591F799234C
:1006400041F78FEF80937002BA9AB99AC19AA0E7E6
:10065000B2E0119698E08E91983018F4392F9927CE
:1006600002C038E09850881FC29808F4C29A00006F
:100670000000C19800000000C19A000000003A95F7
:1006800091F7992341F7B99ABB98C19A98E0A1E7ED
:10069000B2E01196983018F4392F992702C038E04B
:1006A0009850C198000000008894B3990894881F5E
:1006B000C19A000000003A95A1F78E93992351F753
:1006C00000917102003011F40C948503B99ABB9823
:1006D000C19A98E0A1E7B2E01196983018F4392F4A
:1006E000992702C038E09850C19800000000889413
:1006F000B3990894881FC19A000000003A95A1F7A9
:100700008E93992351F70C946003009171020E3F70
:1007100011F40C94AA03B99ABB98C19A98E0A1E786
:10072000B2E01196983018F4392F992702C038E0BA
:100730009850C198000000008894B3990894881FCD
:10074000C19A000000003A95A1F78E93992351F7C2
:100750000C94850381E090E0A4E7B2E08D939C9334
:10076000A4E7B2E00D911C91003052E0150718F09B
:1007700011F00C94EA03B99ABB98C19A98E0A1E7EA
:10078000B2E01196983018F4392F992702C038E05A
:100790009850C198000000008894B3990894881F6D
:1007A000C19A000000003A95A1F78E93992351F762
:1007B00080917102A4E7B2E0AD90BC90AFE6B0E0EA
:1007C000AA0DBB1D8C93A4E7B2E00E948C0A11F025
:1007D0000C94B003B99ABB98C19A98E0A1E7B2E033
:1007E0001196983018F4392F992702C038E09850A4
:1007F000C198000000008894B3990894881FC19A9A
:10080000000000003A95A1F78E93992351F7B99A09
:10081000BB98C19A98E0A1E7B2E01196983018F41D
:10082000392F992702C038E09850C1980000000085
:100830008894B3990894881FC19A000000003A95E3
:10084000A1F78E93992351F7C09A0E9462090895E7
:10085000C09ABA9AB99AC19AA0E7B2E0119698E004
:100860008E91983018F4392F992702C038E09850AB
:10087000881FC29808F4C29A00000000C1980000C6
:100880000000C19A000000003A9591F7992341F7C2
:10089000B99ABB98C19A98E0A1E7B2E01196983056
:1008A00018F4392F992702C038E09850C1980000F9
:1008B00000008894B3990894881FC19A0000000032
:1008C0003A95A1F78E93992351F7C09880E68093CB
:1008D0007002BA9AB99AC19AA0E7B2E0119698E06C
:1008E0008E91983018F4392F992702C038E098502B
:1008F000881FC29808F4C29A00000000C198000046
:100900000000C19A000000003A9591F7992341F741
:10091000BA9AB99AC19AAA81BB81149690E28E9133
:10092000983018F4392F992702C038E09850881F62
:10093000C29808F4C29A00000000C19800000000AC
:10094000C19A000000003A9591F7992341F78FEF83
:1009500080937002BA9AB99AC19AA0E7B2E0119650
:1009600098E08E91983018F4392F992702C038E01A
:100970009850881FC29808F4C29A00000000C198DD
:1009800000000000C19A000000003A9591F79923F9
:1009900041F7BA9AB99AC19AA0E7B2E0119698E0E5
:1009A0008E91983018F4392F992702C038E098506A
:1009B000881FC29808F4C29A00000000C198000085
:1009C0000000C19A000000003A9591F7992341F781
:1009D000B99ABB98C19A98E0A1E7B2E01196983015
:1009E00018F4392F992702C038E09850C1980000B8
:1009F00000008894B3990894881FC19A00000000F1
:100A00003A95A1F78E93992351F700917102003026
:100A100011F40C942A05B99ABB98C19A98E0A1E701
:100A2000B2E01196983018F4392F992702C038E0B7
:100A30009850C198000000008894B3990894881FCA
:100A4000C19A000000003A95A1F78E93992351F7BF
:100A50000C940505C09ABA9AB99AC19AA0E7B2E077
:100A6000119698E08E91983018F4392F992702C08A
:100A700038E09850881FC29808F4C29A000000001D
:100A8000C19800000000C19A000000003A9591F75B
:100A9000992341F7B99ABB98C19A98E0A1E7B2E0CF
:100AA0001196983018F4392F992702C038E09850E1
:100AB000C198000000008894B3990894881FC19AD7
:100AC000000000003A95A1F78E93992351F7C09842
:100AD00081E680937002BA9AB99AC19AA0E7B2E00F
:100AE000119698E08E91983018F4392F992702C00A
:100AF00038E09850881FC29808F4C29A000000009D
:100B0000C19800000000C19A000000003A9591F7DA
:100B1000992341F7BA9AB99AC19AA881B9811496D2
:100B200090E28E91983018F4392F992702C038E05E
:100B30009850881FC29808F4C29A00000000C1981B
:100B400000000000C19A000000003A9591F7992337
:100B500041F78FEF80937002BA9AB99AC19AA0E7D1
:100B6000B2E0119698E08E91983018F4392F9927B9
:100B700002C038E09850881FC29808F4C29A00005A
:100B80000000C19800000000C19A000000003A95E2
:100B900091F7992341F7BA9AB99AC19AA0E7B2E0BE
:100BA000119698E08E91983018F4392F992702C049
:100BB00038E09850881FC29808F4C29A00000000DC
:100BC000C19800000000C19A000000003A9591F71A
:100BD000992341F7B99ABB98C19A98E0A1E7B2E08E
:100BE0001196983018F4392F992702C038E09850A0
:100BF000C198000000008894B3990894881FC19A96
:100C0000000000003A95A1F78E93992351F70091C7
:100C10007102003011F40C942C06B99ABB98C19A59
:100C200098E0A1E7B2E01196983018F4392F99278F
:100C300002C038E09850C198000000008894B39931
:100C40000894881FC19A000000003A95A1F78E937E
:100C5000992351F70C940706C09ABA9AB99AC19A87
:100C6000A0E7B2E0119698E08E91983018F4392FF1
:100C7000992702C038E09850881FC29808F4C29A99
:100C800000000000C19800000000C19A00000000B0
:100C90003A9591F7992341F7B99ABB98C19A98E090
:100CA000A1E7B2E01196983018F4392F992702C0C5
:100CB00038E09850C198000000008894B3990894D7
:100CC000881FC19A000000003A95A1F78E939923DE
:100CD00051F7C09886E680937002BA9AB99AC19A81
:100CE000A0E7B2E0119698E08E91983018F4392F71
:100CF000992702C038E09850881FC29808F4C29A19
:100D000000000000C19800000000C19A000000002F
:100D10003A9591F7992341F700E010E020E030E0A8
:100D2000A0E8B2E00D931D932D933C93BA9AB99A23
:100D3000C19AA0E8B2E0149690E28E91983018F42F
:100D4000392F992702C038E09850881FC29808F4BC
:100D5000C29A00000000C19800000000C19A000083
:100D600000003A9591F7992341F78FEF8093700235
:100D7000BA9AB99AC19AA0E7B2E0119698E08E911A
:100D8000983018F4392F992702C038E09850881FFE
:100D9000C29808F4C29A00000000C1980000000048
:100DA000C19A000000003A9591F7992341F7BA9A49
:100DB000B99AC19AA0E7B2E0119698E08E91983066
:100DC00018F4392F992702C038E09850881FC2982C
:100DD00008F4C29A00000000C19800000000C19A07
:100DE000000000003A9591F7992341F7B99ABB9812
:100DF000C19A98E0A1E7B2E01196983018F4392F23
:100E0000992702C038E09850C198000000008894EB
:100E1000B3990894881FC19A000000003A95A1F781
:100E20008E93992351F700917102003011F00C94C8
:100E30003807B99ABB98C19A98E0A1E7B2E0119639
:100E4000983018F4392F992702C038E09850C1988B
:100E5000000000008894B3990894881FC19A00008C
:100E600000003A95A1F78E93992351F70C9413073C
:100E70000E9462090895C09A8FEF80937002BA9A17
:100E8000B99AC19AA0E7B2E0119698E08E91983095
:100E900018F4392F992702C038E09850881FC2985B
:100EA00008F4C29A00000000C19800000000C19A36
:100EB000000000003A9591F7992341F7B99ABB9841
:100EC000C19A98E0A1E7B2E01196983018F4392F52
:100ED000992702C038E09850C1980000000088941B
:100EE000B3990894881FC19A000000003A95A1F7B1
:100EF0008E93992351F7C09888E580937002BA9A2F
:100F0000B99AC19AA0E7B2E0119698E08E91983014
:100F100018F4392F992702C038E09850881FC298DA
:100F200008F4C29A00000000C19800000000C19AB5
:100F3000000000003A9591F7992341F7BA9AB99ABF
:100F4000C19AA881B981149690E28E91983018F4D4
:100F5000392F992702C038E09850881FC29808F4AA
:100F6000C29A00000000C19800000000C19A000071
:100F700000003A9591F7992341F78FEF8093700223
:100F8000BA9AB99AC19AA0E7B2E0119698E08E9108
:100F9000983018F4392F992702C038E09850881FEC
:100FA000C29808F4C29A00000000C1980000000036
:100FB000C19A000000003A9591F7992341F7BA9A37
:100FC000B99AC19AA0E7B2E0119698E08E91983054
:100FD00018F4392F992702C038E09850881FC2981A
:100FE00008F4C29A00000000C19800000000C19AF5
:100FF000000000003A9591F7992341F7B99ABB9800
:10100000C19A98E0A1E7B2E01196983018F4392F10
:10101000992702C038E09850C198000000008894D9
:10102000B3990894881FC19A000000003A95A1F76F
:101030008E93992351F700917102003011F40C94B2
:101040004008B99ABB98C19A98E0A1E7B2E011961E
:10105000983018F4392F992702C038E09850C19879
:10106000000000008894B3990894881FC19A00007A
:1010700000003A95A1F78E93992351F70C941B0821
:10108000ECE3F6E10E94FB0A0E94B00AAEEABFE080
:10109000E1E7F2E00E94FE0A0E94A80A8EEF809328
:1010A0007002BA9AB99AC19AA0E7B2E0119698E094
:1010B0008E91983018F4392F992702C038E0985053
:1010C000881FC29808F4C29A00000000C19800006E
:1010D0000000C19A000000003A9591F7992341F76A
:1010E00081E090E0A4E7B2E08D939C93A4E7B2E0A6
:1010F0000D911C91003052E0150718F011F00C947E
:10110000A708BA9AB99AC19AAA81BB81119698E0A8
:101110008E91983018F4392F992702C038E09850F2
:10112000881FC29808F4C29A00000000C19800000D
:101130000000C19A000000003A9591F7992341F709
:10114000A4E7B2E00E948C0A11F00C9476088FEFAD
:1011500080937002BA9AB99AC19AA0E7B2E0119648
:1011600098E08E91983018F4392F992702C038E012
:101170009850881FC29808F4C29A00000000C198D5
:1011800000000000C19A000000003A9591F79923F1
:1011900041F7BA9AB99AC19AA0E7B2E0119698E0DD
:1011A0008E91983018F4392F992702C038E0985062
:1011B000881FC29808F4C29A00000000C19800007D
:1011C0000000C19A000000003A9591F7992341F779
:1011D000B99ABB98C19A98E0A1E7B2E0119698300D
:1011E00018F4392F992702C038E09850C1980000B0
:1011F00000008894B3990894881FC19A00000000E9
:101200003A95A1F78E93992351F7009171024FE01F
:101210000423A9E7B2E00C93B99ABB98C19A98E06D
:10122000A1E7B2E01196983018F4392F992702C03F
:1012300038E09850C198000000008894B399089451
:10124000881FC19A000000003A95A1F78E93992358
:1012500051F700917102003011F00C944E09B99AC7
:10126000BB98C19A98E0A1E7B2E01196983018F4C3
:10127000392F992702C038E09850C198000000002B
:101280008894B3990894881FC19A000000003A9589
:10129000A1F78E93992351F70C9429090E94B70A5C
:1012A000E2E4F6E10E94FB0A0E94B00AAEEABFE067
:1012B000E9E7F2E00E94FE0A0E94A80AC09A0E9492
:1012C00062090895C09ABA9AB99AC19AA0E7B2E0A1
:1012D000119698E08E91983018F4392F992702C012
:1012E00038E09850881FC29808F4C29A00000000A5
:1012F000C19800000000C19A000000003A9591F7E3
:10130000992341F7B99ABB98C19A98E0A1E7B2E056
:101310001196983018F4392F992702C038E0985068
:10132000C198000000008894B3990894881FC19A5E
:10133000000000003A95A1F78E93992351F7C098C9
:101340008DE480937002BA9AB99AC19AA0E7B2E08C
:10135000119698E08E91983018F4392F992702C091
:1013600038E09850881FC29808F4C29A0000000024
:10137000C19800000000C19A000000003A9591F762
:10138000992341F700E010E020E030E0A0E8B2E06F
:101390000D931D932D933C93BA9AB99AC19AA0E8E4
:1013A000B2E0149690E28E91983018F4392F992774
:1013B00002C038E09850881FC29808F4C29A000012
:1013C0000000C19800000000C19A000000003A959A
:1013D00091F7992341F78FEF80937002BA9AB99AE7
:1013E000C19AA0E7B2E0119698E08E91983018F477
:1013F000392F992702C038E09850881FC29808F406
:10140000C29A00000000C19800000000C19A0000CC
:1014100000003A9591F7992341F7BA9AB99AC19A7F
:10142000A0E7B2E0119698E08E91983018F4392F29
:10143000992702C038E09850881FC29808F4C29AD1
:1014400000000000C19800000000C19A00000000E8
:101450003A9591F7992341F7B99ABB98C19A90E1CF
:10146000A2E7B2E01296983018F4392F992702C0FB
:1014700038E09850C198000000008894B39908940F
:10148000881FC19A000000003A95A1F78E93992316
:1014900051F7E6E4F6E10E94FB0A0E949A0AAEEADE
:1014A000BFE0E2E7F2E00E94000B0E94920A0E9475
:1014B000A10AC09A089581E090E0A4E7B2E08D937C
:1014C0009C93A4E7B2E00D911C91003052E0150707
:1014D00018F011F00C94810AAEEABFE0E4E7F2E004
:1014E000A190B080EFE6F0E0EA0DFB1D0E94FE0A3D
:1014F0000E94920AA4E7B2E00E948C0A11F00C94B8
:10150000610A0E9462090895481A8827580A0895B6
:10151000480E8827581E0895ED91FC913196FC9352
:10152000EE930895AEEABFE08D91882311F00CD0C0
:10153000FBCF08950E94F10A802D11F005D0FACF5B
:1015400008958DE001D08AE05D9BFECF8CB90895AF
:10155000AEEABFE08D91882311F016D0FBCF08953D
:101560000E94F10A802D11F00FD0FACF089580EC7F
:101570000FC08AEF90E00E94E60A88E309D08EE06F
:1015800007D086E005D00895809300C01CD0089550
:101590008093008018D008953197F1F70895C09A8C
:1015A000B89AC198B99AC298BA9ABB980895C19846
:1015B000C298C0980895C09A0895689462F80895F2
:1015C000E89462F8089581E090E000C0EF93FF9303
:1015D000E8EEF3E03197F1F70197D1F7FF91EF9142
:1015E0000895D8953196002008950F920024039411
:1015F0000BBE0F9008950F920024FACF41E003C074
:1016000042E001C044E0E40F8827F81F8291982F40
:10161000829506D0892F04D04A95C1F70C94170BF8
:101620008F708A3008F0895F805D8D9308958827D8
:101630008D93089543303A0043313A004332343AAF
:0E164000000057723A005374617475733A00DB
:00000001FF
